:020000040000FA
:10300000DEEF25F0E4EF25F0EAEF25F0F9EF25F00B
:10301000FAEF25F000EF26F03CEF26F04BEF26F01C
:103020002CEF26F034EF26F05AEF26F024EF26F0AE
:103030001EEF26F006EF26F011EF26F080EF19F0D4
:1030400081EF19F082EF19F083EF19F02BEF26F0E2
:103050002AEF26F084EF19F085EF19F086EF19F0CA
:103060001200000012000000120000001200000018
:103070001200000012000000120000001200000008
:10308000FFFFFFFFFFFFFFFFFFFFFFFFFFFFFFFF50
:10309000FFFFFFFFFFFFFFFFFFFFFFFFFFFFFFFF40
:103300001200120012001200120012001200D9CF97
:10331000EDFFE9CFD9FF10C0EDFF11C0EDFF12C0E6
:10332000EDFF13C0EDFF14C0EDFF106E020EDBCFFA
:1033300011F010C081F000018951010A05E111501E
:10334000ED6EC0EC24F0E92A00018951020A2DE15A
:10335000100E88EC16F0000EED6E400EED6E360E7F
:10336000B2EC2CF0020EE926105090EC16F0136A25
:10337000D8901034126E13363E0E12263E0E1322D3
:10338000000E146A1422122AD8B0132AD8B0142AB4
:1033900012C0F6FF13C0F7FF14C0F8FF0900F5CF05
:1033A000F2F00001F25194EC16F000018951040A88
:1033B00007E1115003E0E7EC26F002D064EC26F0C0
:1033C00000019051D8B44ED01150D8B44BD0105009
:1033D000110A19E01050190A1AE010501D0A20E0D5
:1033E0001050210A20E01050230A20E01050270A34
:1033F00039E01050290A24E010502F0A27E010501D
:10340000360A2EE02FD0E1EC27F07CEF1CF0000E06
:10341000ED6E54EC23F0E92A0001906B7CEF1CF078
:103420006FEC29F01FD00AEC2BF01CD0000EED6ED3
:10343000400EED6E380EB2EC2CF0020EE92612D0E2
:1034400054EC20F00001906B7CEF1CF0000EED6E50
:10345000400EED6E3E0EB2EC2CF0020EE92602D0CC
:1034600012EC24F000018D5109E0115005E01050DC
:10347000ED6E54EC23F0E92A7CEF1CF000018C5136
:1034800006E0115002E054EC20F07CEF1CF01050EC
:1034900001E170D01050010A02E17CEF1CF01050E5
:1034A000020A01E172D01050030A01E188D01050E5
:1034B000040A01E19ED01050050A01E1A9D0105084
:1034C000060A01E1B4D01050070A01E1BFD0105044
:1034D0000C0A01E1CAD010500E0A02E17CEF1CF088
:1034E00010500F0A02E17CEF1CF01050100A01E1AD
:1034F000C3D01050140A01E1D4D01050180A01E1D1
:10350000E4D010501C0A01E1EAD01050200A01E179
:10351000F0D01050240A01E1F6D01050280A01E141
:10352000FCD010502C0A01E102D11050300A01E108
:1035300008D11050330A01E117D11050340A01E1CB
:1035400025D11050380A01E131D110503A0A01E179
:103550003CD110503B0A01E14AD110503C0A01E134
:1035600061D110503E0A01E17BD110503F0A01E1C8
:10357000B2D1C2D100019151D8B4BED100018E5157
:10358000D8B4BAD1D2EC16F0B7D11150D8A4B4D176
:10359000AF0E00018225106E126A000E122210C0BA
:1035A000E1FF12C0E2FFE7CF13F0132A10C0E1FFE2
:1035B00012C0E2FF13C0E7FF1FEC29F09DD11150AC
:1035C000D8A49AD1AF0E00018225106E126A000EA7
:1035D000122210C0E1FF12C0E2FFE7CF13F0130682
:1035E00010C0E1FF12C0E2FF13C0E7FF1FEC29F09B
:1035F00083D100018E5106E1000EED6E6BEC2CF0D4
:10360000E92A7AD1300EED6E6BEC2CF0E92A74D1F8
:1036100000018E5106E10C0EED6E6BEC2CF0E92AE8
:103620006BD13C0EED6E6BEC2CF0E92A65D10001FC
:103630008E5106E1180EED6E6BEC2CF0E92A5CD190
:10364000480EED6E6BEC2CF0E92A56D100018E513C
:1036500006E1240EED6E6BEC2CF0E92A4DD1540EF0
:10366000ED6E6BEC2CF0E92A47D182EC16F050ECB1
:103670002CF09BEC2BF040D100018E51D8B43CD102
:103680004DEC2EF0106EFF0E105CD8B035D14DEC25
:103690002EF0106E102A1050ED6EEAEC2BF0E92A95
:1036A0002BD100018E5111E04DEC2EF0106E310E39
:1036B000105CD8A021D14DEC2EF0106E10061050E9
:1036C000ED6EEAEC2BF0E92A17D100019051D8B445
:1036D00013D1080E0001826FB7EC29F00DD1000163
:1036E0009051D8B409D1090E0001826FB7EC29F0CE
:1036F00003D100019051D8B4FFD0060E0001826FB3
:10370000B7EC29F0F9D000019051D8B4F5D0070EEC
:103710000001826FB7EC29F0EFD000019051D8B4CE
:10372000EBD0040E0001826FB7EC29F0E5D0000168
:103730009051D8B4E1D0050E0001826FB7EC29F0AA
:10374000DBD00001905106E0020E0001826FB7EC61
:1037500029F0D2D000019151D8B4CED01150D8B4B4
:10376000CBD051EC28F0C8D0115003E000018E6B93
:10377000C3D0010E00018E6F000EED6E400EED6E97
:10378000440EB2EC2CF0020EE926B6D000019151A5
:1037900003E0040E0001896F00019051D8B4ACD051
:1037A000030E0001826FB7EC29F0A6D00001915101
:1037B00003E0010E0001896F00019051D8B49CD044
:1037C0000001826BB7EC29F097D0115003E00001A3
:1037D000906B92D0010E0001906F000EED6E400EC6
:1037E000ED6E4A0EB2EC2CF0020EE92685D0115097
:1037F000D8B482D0100E88EC16F000018B5106E18F
:10380000010E00018B6F55EC2DF076D0000EED6EA1
:10381000400EED6E500EB2EC2CF0020EE926CDEC0F
:103820002CF06AD00001915111E0020E0001896F65
:10383000000EED6E400EED6E560EB2EC2CF0020E48
:10384000E926000189518EEC16F056D00001905106
:10385000D8B452D0010E0001826FB7EC29F04CD0E1
:10386000115005E00001916B9BEC2BF045D0010E4F
:103870000001916F000E88EC16F0000EED6E400E08
:10388000ED6E620EB2EC2CF0020EE926400E88ECD2
:1038900016F0000EED6E400EED6E720EB2EC2CF0D6
:1038A000020EE926800E88EC16F0000EED6E400E3A
:1038B000ED6E820EB2EC2CF0020EE926C00E88EC02
:1038C00016F0000EED6E400EED6E920EB2EC2CF086
:1038D000020EE92611D011500DE1000EED6E400EE2
:1038E000ED6EA20EB2EC2CF0020EE926010E0001E4
:1038F000926F02D00001926BECCF14F0ECCF13F07A
:10390000ECCF12F0ECCF11F0ECCF10F0ECCFD9FFF0
:10391000120010C0EDFF11C0EDFF12C0EDFF13C08B
:10392000EDFF14C0EDFF15C0EDFF16C0EDFF17C091
:10393000EDFF18C0EDFF19C0EDFF1AC0EDFF1BC071
:10394000EDFF1CC0EDFF1DC0EDFF1EC0EDFF1FC051
:10395000EDFF20C0EDFF21C0EDFF00018951040AF9
:1039600002E196EC22F000018651180A02E1000102
:10397000866B000186510DE000018651060A09E0C0
:10398000000186510C0A05E000018651120A01E08F
:103990009FD100018751100A08E10001876B0001E7
:1039A000852B040E855D01E3856B0001875101E0E5
:1039B000A3D0106A116A126A136A146A156A166A29
:1039C0000A0E105CD8B098D0105003E1400E88EC7D
:1039D00016F01050050A03E1800E88EC16F03E0E3A
:1039E0001124176E3D0E1220186E196A000E19224E
:1039F00085C01AF01B6A1A5017261B501822E86A55
:103A0000192217C0F6FF18C0F7FF19C0F8FF090008
:103A1000F5CF17F0175098EC16F0105000018219EE
:103A20001FE13C0E94EC16F03E0E1124176E3D0E75
:103A300012201A6E1B6A000E1B2285C01CF01D6A24
:103A40001C5017261D501A22E86A1B2217C0F6FFC9
:103A50001AC0F7FF1BC0F8FF0900F5CF83F003D0B1
:103A6000200E94EC16F03E0E1524176E3D0E162017
:103A70001A6E1B6A000E1B2285C01CF01D6A1C50AA
:103A800017261D501A22E86A1B2217C0F6FF1AC01B
:103A9000F7FF1BC0F8FF0900F5CF17F0176601D03C
:103AA0001DD01750400DF3CF17F0F4CF1AF0400E91
:103AB0001A26000E13241B6E010E14201C6E800E9D
:103AC0001D6E1D50ED6E1C50ED6E1B50ED6E1A50AC
:103AD000ED6E175022EC2DF0040EE926040E11268F
:103AE000D8B0122A100E1326D8B0142A040E1526A8
:103AF000D8B0162A102A64D70001885188EC16F035
:103B000000018651060A04E1000E94EC16F003D081
:103B1000010E94EC16F00001875188EC16F0020EAD
:103B200094EC16F0106A116A126A136A146A100E85
:103B3000105CD8B0C9D0000E1124156E010E1220F1
:103B4000166E87C017F01A6A175015261A501622DB
:103B500015C0E1FF16C0E2FFE7CF15F01550800A4F
:103B600034E1CF0E1024166E176A000E172216C00D
:103B7000E1FF17C0E2FFE7CF16F0166601D09AD03A
:103B8000900E1024166E165024EC16F0CF0E102452
:103B9000166E1A6A000E1A2216C0E1FF1AC0E2FF62
:103BA000E7CF16F0165024EC16F0000E24EC16F0B9
:103BB000CF0E1024166E1B6A000E1B2216C0E1FFEA
:103BC0001BC0E2FF000EE76E75D01550810A01E1BF
:103BD00071D0CF0E1024156E166A000E162215C075
:103BE000E1FF16C0E2FFE7CF15F0156601D024D043
:103BF000900E1024156E155024EC16F0CF0E1024E4
:103C0000156E1B6A000E1B2215C0E1FF1BC0E2FFF0
:103C1000E7CF15F0155024EC16F0000E24EC16F04A
:103C2000CF0E1024156E1C6A000E1C2215C0E1FF79
:103C30001CC0E2FF000EE76E900E1024156E1550AA
:103C400024EC16F0000E1324156E010E14201C6EC9
:103C500087C01DF01E6A1D5015261E501C2215C05F
:103C6000E1FF1CC0E2FFE7CF15F0155024EC16F081
:103C70007F0E24EC16F0CF0E1024156E1D6A000E78
:103C80001D22000E13241E6E010E14201F6E87C00D
:103C900020F0216A20501E2621501F221EC0E1FF65
:103CA0001FC0E2FFE7CF1EF015C0E1FF1DC0E2FF1D
:103CB0001EC0E7FF100E1126D8B0122A100E1326D0
:103CC000D8B0142A102A33D787C088F00001872B78
:103CD0000001862BECCF21F0ECCF20F0ECCF1FF0D1
:103CE000ECCF1EF0ECCF1DF0ECCF1CF0ECCF1BF0B6
:103CF000ECCF1AF0ECCF19F0ECCF18F0ECCF17F0B6
:103D0000ECCF16F0ECCF15F0ECCF14F0ECCF13F0B5
:103D1000ECCF12F0ECCF11F0ECCF10F0120000005D
:103D200000001F1F1F1F000000001F11111F1F0E8A
:103D300004001F1F1F1F1F0E04001F11111F000072
:103D40000000000000000000000000000000000073
:103D50000000000000000000000000000000000063
:103D600000000A0B0C0D0000000000000000000025
:103D70000000000000000000000000000000596189
:103D80006D6168612046533152004D41747269780B
:103D900020313030300059616D6168612046533107
:103DA0005200556E757365642063686E3400536904
:103DB0006450686F6E653120200053696450686FED
:103DC0006E65322020004A554E4F2031303620207B
:103DD00020004D415452495820313030300042616A
:103DE000737353546174696F6E004472756D5354EC
:103DF0006174696F6E00556E757365642063683118
:103E00003100556E75736564206368313200556EFC
:103E100075736564206368313300556E757365642E
:103E2000206368313400556E7573656420636831B2
:103E30003500556E75736564206368313600803FC8
:103E4000803F803F803F803F803F803F803F2024F5
:103E50001F2A805D103F803F213F803D803F802BA7
:103E60001C500D4C0C3C1E2D1D400F5B0E3E193995
:103E700018490A4A094E1B301A4F804B0B4D163712
:103E80001559064705568038175508480742123518
:103E900011520344025814361354804604430F331E
:103EA0000E578041803F803410450153005A8031C5
:103EB000803F803F803F0D320C51803F8020432D5A
:103EC00000432300442D00442300452D00462D00CF
:103ED000462300472D00472300412D004123004287
:103EE0002D001011B15BB15BB15BB15BB15BB15B3C
:103EF0000102696AB15BB15BB15BB15BB15BB15BA4
:103F0000B15B50470000282E5F5F5F2F292048419A
:103F100052440000283D5E2E5E3D2920545241430C
:103F20004B4552002822292D2822292000004D49E6
:103F30004449204D45524745522044495341424C43
:103F4000454400004D494449204D455247455220C3
:103F5000454E41424C4544004D42204C696E6B2019
:103F6000456E6420506F696E74004D42204C696E3E
:103F70006B2046776420506F696E74004552524F33
:103F800052004E554C0050414400494E505554206B
:103F900000004F4B20202020200050524700424E6E
:103FA0004B002B00524E443A000020524543000083
:103FB00050004F4B00005061747465726E004241B6
:103FC0004E4B535449434B2030780000577269746C
:103FD0006520706872617365203078005361766582
:103FE000204F4B0042797465206D69736D61746375
:103FF00068004E6F2042616E6B537469636B000002
:1040000053617665206572726F72000042414E4BBB
:104010004C4F41440000415250002053544F500037
:1040200050687261736500002043433A0000202D00
:104030002000203078002300506173740000436F2B
:10404000707900005348465400004354524C00001D
:1040500053544F5000005B44454255475D4D4F441B
:104060004500313A504C4159202020353A534156B1
:104070004500323A44454255472020363A454449A6
:104080005400333A4D455247455220373A41494E44
:104090000000343A41525045472020383A4D4F4EA7
:1040A000000053504143000010C0EDFF11C0EDFF70
:1040B00012C0EDFF13C0EDFF14C0EDFF15C0EDFF02
:1040C00016C0EDFF17C0EDFF00018C510AE10001A1
:1040D0008D6B010E00018C6F0001946B65EC27F075
:1040E0004DD100018151010A19E100018251100DE9
:1040F000F3CF10F0F4CF11F0000E1026010E1122B4
:1041000094C012F0136A125010261350112210C0DE
:10411000E1FF11C0E2FF810EE76EFCD0000181518A
:10412000020A26E10001942B100E945D01E3946BCA
:1041300065EC27F000018251100DF3CF10F0F4CFA1
:1041400011F0000E1026010E112294C012F0136A15
:10415000125010261350112210C0E1FF11C0E2FFCF
:10416000E7CF10F01050ED6EBAEC28F0E92A06D136
:1041700000018151030A28E10001945103E1100E6E
:104180000001946F0001940765EC27F00001825153
:10419000100DF3CF10F0F4CF12F0000E1026010E28
:1041A000122294C013F0146A1350102614501222D5
:1041B00010C0E1FF12C0E2FFE7CF10F01050ED6E2B
:1041C000BAEC28F0E92ADAD0000181510C0A01E0AA
:1041D00040D0106A100E105C1AE200018251100DDE
:1041E000F3CF13F0F4CF14F0000E1326010E1422B7
:1041F00010C015F0166A155013261650142213C05D
:10420000E1FF14C0E2FF800EE76E102AE3D7000141
:10421000946B65EC27F000018251100DF3CF10F084
:10422000F4CF13F0000E1026010E132294C014F0E8
:10423000156A145010261550132210C0E1FF13C048
:10424000E2FFE7CF10F01050ED6EBAEC28F0E92A4B
:1042500095D000018151390A05E100018C6B9BEC7E
:104260002BF08CD0000181513B0A01E153D00001B9
:1042700081513F0A19E100018251100DF3CF10F076
:10428000F4CF14F0000E1026010E142294C015F085
:10429000166A155010261650142210C0E1FF14C0E3
:1042A000E2FF800EE76E36D0146AD89000018135A7
:1042B000106E14363E0E10263E0E1422000E156AA5
:1042C000152210C0F6FF14C0F7FF15C0F8FF090053
:1042D000F5CF10F01050800A01E150D0000182515A
:1042E000100DF3CF14F0F4CF15F0000E1426010ECC
:1042F000152294C016F0176A16501426175015226E
:104300008AC016F01650102614C0E1FF15C0E2FF57
:1043100010C0E7FF0001942B65EC27F000018251EB
:10432000100DF3CF10F0F4CF14F0000E1026010E94
:10433000142294C015F0166A155010261650142237
:1043400010C0E1FF14C0E2FFE7CF10F01050ED6E97
:10435000BAEC28F0E92A100E0001945D0FE382EC1C
:1043600016F0000EED6E3F0EED6EB20EB2EC2CF0BC
:10437000020EE92600018C6B0001946BECCF17F064
:10438000ECCF16F0ECCF15F0ECCF14F0ECCF13F02F
:10439000ECCF12F0ECCF11F0ECCF10F01200D9CF2F
:1043A000EDFFE9CFD9FF10C0EDFF11C0EDFF12C046
:1043B000EDFF13C0EDFF14C0EDFF15C0EDFF16C0FB
:1043C000EDFF17C0EDFF18C0EDFF106E800E88ECFA
:1043D00016F01050070A16E1000EED6E400EED6E5D
:1043E000200EB2EC2CF0020EE926105038EC16F03C
:1043F000116E115098EC16F0105038EC16F00001C8
:10440000836F7FD010508EEC16F0000EED6E400ED4
:10441000ED6E280EB2EC2CF0020EE926126AD8904E
:1044200000018235116E1236E20E11263E0E122266
:10443000000E136A132210C014F0156A14501126CE
:1044400015501222E86A132211C0F6FF12C0F7FFBE
:1044500013C0F8FF0900F5CF11F0115098EC16F0D9
:10446000000EED6E400EED6E2E0EB2EC2CF0020E34
:10447000E926105038EC16F0116E115092EC16F03F
:10448000000EED6E400EED6E320EB2EC2CF0020E10
:10449000E926105038EC16F0116E115098EC16F019
:1044A000020E105C2EE2B00E00018225116E11503A
:1044B00024EC16F0166AD89000018235116E16367B
:1044C000E20E11263E0E1622000E176A1722115018
:1044D0001426165015221750186A182214C0F6FF19
:1044E00015C0F7FF18C0F8FF0900F5CF14F01450FD
:1044F00024EC16F0105038EC16F0106E105024EC2E
:1045000016F0ECCF18F0ECCF17F0ECCF16F0ECCFA4
:1045100015F0ECCF14F0ECCF13F0ECCF12F0ECCFA1
:1045200011F0ECCF10F0ECCFD9FF120010C0EDFF6E
:1045300011C0EDFF12C0EDFF13C0EDFF14C0EDFF81
:10454000C00E88EC16F0000EED6E400EED6E160EED
:10455000B2EC2CF0020EE9260001965120E1000198
:10456000956B000EED6E400EED6E1A0EB2EC2CF057
:10457000020EE9260001986701D010D0900E0001CC
:104580008225106E105024EC16F00001985124EC96
:1045900016F0000E24EC16F00001986B7AD00001A2
:1045A000972B030E975DD8A074D0976B0001986786
:1045B00001D010D0900E00018225106E105024EC16
:1045C00016F00001985124EC16F0000E24EC16F0C1
:1045D0000001986BDF0E00019525106E116A000E28
:1045E000112210C0E1FF11C0E2FFE7CF10F010660A
:1045F00001D02AD0105092EC16F0900E00018225C6
:10460000106E105024EC16F0DF0E00019525106E90
:10461000116A000E112210C0E1FF11C0E2FFE7CFC6
:1046200010F0105024EC16F07F0E24EC16F0DF0E84
:1046300000019525106E126A000E122210C0E1FFD3
:1046400012C0E2FFE7CF98F096C010F0126AFF0E9A
:104650001026D8A0120695C013F0146A1450800FCB
:10466000F36E1250800FF35C02E11050135C03E311
:10467000010E0001996F010E0001955D02E200013B
:10468000996B0001995103E10001952B02D00001C3
:104690009507ECCF14F0ECCF13F0ECCF12F0ECCF89
:1046A00011F0ECCF10F01200D9CFEDFFE9CFD9FF18
:1046B00010C0EDFF11C0EDFF12C0EDFF13C0EDFF04
:1046C000020EDBCF10F000018D511DE182EC16F0DF
:1046D000020E0001896F010E00018D6F0001936BC6
:1046E000116A100E115C0EE2BF0E1124126E136AD5
:1046F000000E132212C0E1FF13C0E2FF000EE76EAE
:10470000112AEFD784D0000E88EC16F0000EED6E63
:104710003F0EED6E8A0EB2EC2CF0020EE92600017F
:104720009329116E115090EC16F0105007E01050C4
:10473000010A29E01050390A32E034D000019367B1
:1047400001D065D000019307BF0E9325116E126A48
:10475000000E122211C0E1FF12C0E2FF000EE76E50
:10476000400E9325116E115088EC16F0BD0EF66EBA
:104770003E0EF76E000EF86E0900F5CF11F01150E5
:1047800094EC16F044D0000EED6E3F0EED6E920EDE
:10479000B2EC2CF0020EE92600018D6B38D000013E
:1047A0008D6B35D0400E00019325116E115088ECB1
:1047B00016F0BF0E00019325116E126A000E122230
:1047C00011C0E1FF12C0E2FF10C0E7FF116AD890EC
:1047D000103611363E0E10263E0E1122000E126AC1
:1047E0001222102AD8B0112AD8B0122A10C0F6FF0F
:1047F00011C0F7FF12C0F8FF0900F5CF10F01050FC
:1048000094EC16F0100E0001935D01E2932BECCFB7
:1048100013F0ECCF12F0ECCF11F0ECCF10F0ECCFA6
:10482000D9FF120010C0EDFF11C0EDFF12C0EDFF67
:1048300013C0EDFF14C0EDFF0001835101E195D0DD
:10484000000E88EC16F0000EED6E3F0EED6EBE0E03
:10485000B2EC2CF0020EE926F0EC16F0106E1050BF
:1048600098EC16F0400E88EC16F0000EED6E3F0E40
:10487000ED6ECC0EB2EC2CF0020EE9260001835155
:1048800098EC16F0800E88EC16F000018351400D74
:10489000F3CF10F0F4CF11F0400E11260001825139
:1048A000100DF3CF12F0F4CF13F0000E1226010E0C
:1048B0001322800E146E1450ED6E1350ED6E1250D4
:1048C000ED6E1150ED6E105017EC2DF0106E040EC1
:1048D000E926030E105CD8B03FD015C0EDFF16C01E
:1048E000EDFF166A10341636E8341636FC0B156EDA
:1048F000000EFB6E490EFA6E100E15261650FA22A7
:10490000D8B0FB2A1550ECCF16F0ECCF15F0F96EAD
:104910008EEF24F098EF24F0A2EF24F0000EED6E5D
:104920003F0EED6EDC0EB2EC2CF0020EE9261DD02F
:10493000000EED6E3F0EED6EE40EB2EC2CF0020EAA
:10494000E92613D0000EED6E3F0EED6EF20EB2ECC6
:104950002CF0020EE92609D0000EED6E400EED6E31
:10496000000EB2EC2CF0020EE926ECCF14F0ECCFE6
:1049700013F0ECCF12F0ECCF11F0ECCF10F01200EE
:10498000D9CFEDFFE9CFD9FF10C0EDFF11C0EDFF8A
:1049900012C0EDFF13C0EDFF14C0EDFF15C0EDFF19
:1049A00016C0EDFF17C0EDFF020EDBCF10F00001C7
:1049B000905101E066D0126AD89000018135116EE5
:1049C00012363E0E11263E0E1222000E136A1322DC
:1049D00011C0F6FF12C0F7FF13C0F8FF0900F5CFB2
:1049E00011F01150800A01E14CD0900E0001822597
:1049F000116E115024EC16F0146AD8900001813524
:104A0000116E14363E0E11263E0E1422000E156A4B
:104A1000152211C0F6FF14C0F7FF15C0F8FF0900FA
:104A2000F5CF11F08AC016F016501126115024EC63
:104A300016F0105002E0106A02D07F0E106E105077
:104A400024EC16F0116AD89000018135106E1136F1
:104A50003E0E10263E0E1122000E166A162210C0BF
:104A6000F6FF11C0F7FF16C0F8FF0900F5CF10F0F0
:104A70008AC017F0175010261050ED6EBAEC28F0CF
:104A8000E92AECCF17F0ECCF16F0ECCF15F0ECCF15
:104A900014F0ECCF13F0ECCF12F0ECCF11F0ECCF20
:104AA00010F0ECCFD9FF120010EE9FF0080EF36E5D
:104AB000E668F32EFDD710EEA7F0080EF36EE66A57
:104AC000F32EFDD7000EC4EC16F0036E000E68EC5A
:104AD00016F000019D6B120000019D29070BC4EC2C
:104AE00016F0036E000E68EC16F01200000E5CEC7F
:104AF00016F010EE9FF000019D51E3CF0BF003C0C4
:104B0000E3FF10EEA7F09D51E1260B500318E712CA
:104B10009D29070B9D6F120000019E6B10EEA7F000
:104B20009E51E126E75010E0E7B013D8E7B214D861
:104B3000E7B415D8E7B616D8E7B817D8E7BA18D843
:104B4000E7BC19D8E7BE1AD89E2B070E9E65E6D79C
:104B50001200E790000E14D0E792010E11D0E794F6
:104B6000020E0ED0E796030E0BD0E798040E08D085
:104B7000E79A050E05D0E79C060E02D0E79E070EC9
:104B80009B6F10EE9FF09E51E1269B51C6EC16F0F4
:104B9000E714D8A4010E9C6F046E9E519A6F080D05
:104BA000F3509B25036E9CC0EDFF87EC19F0E92ABA
:104BB00010EEA7F000019E51E126120003EE7FF0F7
:104BC00023EE7FF06FEF2BF003EE7FF023EE7FF00C
:104BD0003DEF2EF023EE3FF0E9CFDDFFEACFDDFF22
:104BE00003EE3DF04AEC2EF03FC3E9FF3EC3EAFF7F
:104BF0001200120003EE7FF023EE7FF038EF2EF06C
:104C000003EE7FF023EE7FF0C4EF2BF003EE7FF096
:104C100023EE7FF005C0EDFF04C0EDFF0350E0EF91
:104C20002DF003EE7FF023EE7FF005C0EDFF04C012
:104C3000EDFF03C0EDFFED6ED9EF2DF003EE7FF039
:104C400023EE7FF055EF2EF003EE7FF023EE7FF0A2
:104C5000D2EF2DF01200120003EE7FF023EE7FF072
:104C600004C0EDFFCBEF2DF003EE7FF023EE7FF0DD
:104C700004C0EDFFC4EF2DF023EE3FF0E9CFDDFFE0
:104C8000EACFDDFF03EE3DF085EC2CF03FC3E9FFFA
:104C90003EC3EAFF120023EE3FF0E9CFDDFFEACF8B
:104CA000DDFF03EE3DF047EC2EF03FC3E9FF3EC3CE
:104CB000EAFF120003EE7FF023EE7FF005C0EDFF68
:104CC00004C0EDFFCFEF21F010C0EDFF11C0EDFFEC
:104CD00012C0EDFF13C0EDFF14C0EDFF15C0EDFFD6
:104CE00016C0EDFF17C0EDFF18C0EDFF116AD89098
:104CF00000018135106E11363E0E10263E0E112237
:104D0000000E126A122210C0F6FF11C0F7FF12C087
:104D1000F8FF0900F5CF10F08AC013F010501326E9
:104D20001050800A01E140D0DF0E00019625106E80
:104D3000146A000E142210C0E1FF14C0E2FF13C079
:104D4000E7FF96C010F0962B020E965D2DE3010E44
:104D5000105C2AE3DF0E1024136E146A000E142276
:104D600013C0E1FF14C0E2FFE7CF15F01004166E88
:104D7000DF0E1626000E176A172216C0E1FF17C0B5
:104D8000E2FFE7CF18F01850155C0CE216C0E1FF07
:104D900017C0E2FF15C0E7FF13C0E1FF14C0E2FF38
:104DA00018C0E7FF1006D3D7ECCF18F0ECCF17F000
:104DB000ECCF16F0ECCF15F0ECCF14F0ECCF13F0F5
:104DC000ECCF12F0ECCF11F0ECCF10F0120010C0CD
:104DD000EDFF11C0EDFF12C0EDFF13C0EDFF14C0D9
:104DE000EDFF15C0EDFF16C0EDFF17C0EDFF18C0B9
:104DF000EDFF116AD89000018135106E11363E0E1C
:104E000010263E0E1122000E126A122210C0F6FF6A
:104E100011C0F7FF12C0F8FF0900F5CF10F01050D5
:104E2000800A01E13FD0116A00019651115C38E21D
:104E3000DF0E1124126E136A000E132212C0E1FF5E
:104E400013C0E2FFE7CF14F010C015F0166A10BED1
:104E500016068AC017F0186A175015261850162221
:104E6000176A1750800FF36E1650800FF35C02E143
:104E70001550145C13E31128146EDF0E1426000E77
:104E8000156A152214C0E1FF15C0E2FFE7CF14F048
:104E900012C0E1FF13C0E2FF14C0E7FF112AC4D71C
:104EA00000019607ECCF18F0ECCF17F0ECCF16F01E
:104EB000ECCF15F0ECCF14F0ECCF13F0ECCF12F0F8
:104EC000ECCF11F0ECCF10F0120010C0EDFF11C0CC
:104ED000EDFF12C0EDFF82EC16F0000E88EC16F02C
:104EE000000E94EC16F0010E94EC16F0010E94EC0A
:104EF00016F0010E94EC16F0000E94EC16F0010E74
:104F000094EC16F0010E94EC16F0010E94EC16F0F1
:104F1000000E94EC16F0010E94EC16F0010E94ECD9
:104F200016F0010E94EC16F0000E94EC16F0010E43
:104F300094EC16F0010E94EC16F0010E94EC16F0C1
:104F4000000EED6E3F0EED6EAA0EB2EC2CF0020ECE
:104F5000E9260001945188EC16F0020E94EC16F04C
:104F6000910E88EC16F0000EED6E3F0EED6EB00E59
:104F7000B2EC2CF0020EE9260001835198EC16F0F9
:104F8000C00E88EC16F0000182510C0DF3CF10F02A
:104F9000F4CF11F07E0E10263D0E1122000E126A83
:104FA00012221250ED6E1150ED6E1050B2EC2CF03A
:104FB000020EE926ECCF12F0ECCF11F0ECCF10F09E
:104FC000120010C0EDFF11C0EDFF12C0EDFF13C0C5
:104FD000EDFF14C0EDFF15C0EDFF16C0EDFF17C0CB
:104FE000EDFFCDEC2CF082EC16F0000EED6E3F0ED6
:104FF000ED6EB60EB2EC2CF0020EE92600018451E3
:1050000098EC16F0106A116A126A100E105C38E201
:10501000105003E1400E88EC16F01050050A03E131
:10502000800E88EC16F010500A0A03E1C00E88ECDE
:1050300016F03E0E1124136E3D0E1220146E156AEA
:10504000000E152284C016F0176A1650132617504A
:105050001422E86A152213C0F6FF14C0F7FF15C02A
:10506000F8FF0900F5CF13F0135098EC16F0200E5E
:1050700094EC16F0040E1126D8B0122A102AC5D7C7
:10508000ECCF17F0ECCF16F0ECCF15F0ECCF14F01E
:10509000ECCF13F0ECCF12F0ECCF11F0ECCF10F01E
:1050A000120010C0EDFF000E88EC16F012EC16F0A6
:1050B000106E040E105CD8B051D011C0EDFF12C0BC
:1050C000EDFF126A10341236E8341236FC0B116E02
:1050D000000EFB6E500EFA6EF00E11261250FA22E0
:1050E000D8B0FB2A1150ECCF12F0ECCF11F0F96ED2
:1050F00080EF28F08DEF28F09AEF28F0A4EF28F049
:10510000010E14EC16F0000EED6E3F0EED6E2E0E3D
:10511000B2EC2CF0020EE9262AD0000E14EC16F0A8
:10512000000EED6E3F0EED6E440EB2EC2CF0020E52
:10513000E9261DD0000EED6E3F0EED6E580EB2EC5E
:105140002CF0020EE92613D0000EED6E3F0EED6E30
:105150006A0EB2EC2CF0020EE92609D0000EED6EBC
:105160003F0EED6E7C0EB2EC2CF0020EE926ECCF79
:1051700010F01200D9CFEDFFE9CFD9FF10C0EDFF3D
:1051800011C0EDFF12C0EDFF13C0EDFF020EDBCF2B
:1051900010F01050800A0DE1510E88EC16F0000E50
:1051A000ED6E3F0EED6E820EB2EC2CF0020EE92693
:1051B0003BD01050810A0DE1510E88EC16F0000E24
:1051C000ED6E3F0EED6E860EB2EC2CF0020EE9266F
:1051D0002BD0116A126A0C0E1226112A1250105C82
:1051E000FAE21106510E88EC16F011500C0DF3CFB7
:1051F00012F01250105E1050030DF3CF10F0F4CFE8
:1052000012F0BE0E10263E0E1222000E136A13225A
:105210001350ED6E1250ED6E1050B2EC2CF0020EE9
:10522000E92611508EEC16F0ECCF13F0ECCF12F013
:10523000ECCF11F0ECCF10F0ECCFD9FF120010C082
:10524000EDFF11C0EDFF12C0EDFF0E0E88EC16F061
:10525000000EED6E3F0EED6E9A0EB2EC2CF0020ECB
:10526000E926AF0E00018225106E116A000E112290
:1052700010C0E1FF11C0E2FFE7CF12F0800E125C18
:1052800006E310C0E1FF11C0E2FF000EE76E10C0A0
:10529000E1FF11C0E2FFE7CF10F0102A105092ECAE
:1052A00016F0C00E00018225106E105024EC16F08E
:1052B000AF0E00018225106E126A000E122210C07D
:1052C000E1FF12C0E2FFE7CF10F0105024EC16F01F
:1052D000ECCF12F0ECCF11F0ECCF10F0120010C0B8
:1052E000EDFF11C0EDFF12C0EDFF13C0EDFF14C0C4
:1052F000EDFF0001835130E0000EED6E400EED6ECB
:105300000C0EB2EC2CF0020EE9260001835198EC51
:1053100016F000018351400DF3CF10F0F4CF11F0DF
:10532000400E112600018251100DF3CF12F0F4CF80
:1053300013F0000E1226010E1322800E146E14506C
:10534000ED6E1350ED6E1250ED6E1150ED6E10506B
:1053500022EC2DF0040EE926ECCF14F0ECCF13F084
:10536000ECCF12F0ECCF11F0ECCF10F0120010C027
:10537000EDFF11C0EDFF12C0EDFF13C0EDFF8F0E6A
:1053800088EC16F0000EED6E3F0EED6E020EB2ECE4
:105390002CF0020EE926AF0E00018225106E116A74
:1053A000000E112210C0E1FF11C0E2FFE7CF10F0A4
:1053B000102A105092EC16F0C00E88EC16F0000186
:1053C00082510C0DF3CF10F0F4CF12F07E0E1026A8
:1053D0003D0E1222000E136A13221350ED6E12506E
:1053E000ED6E1050B2EC2CF0020EE926ECCF13F06B
:1053F000ECCF12F0ECCF11F0ECCF10F0120010C097
:10540000EDFF11C0EDFF12C0EDFF13C0EDFF14C0A2
:10541000EDFF15C0EDFF16C0EDFF17C0EDFF106AE0
:10542000116A126A100E105C1FE2000E1124136E36
:10543000010E1220146E156A100E155C0FE215C0D5
:1054400016F0176A135016261450172216C0E1FFE3
:1054500017C0E2FF800EE76E152AEED7100E112658
:10546000D8B0122A102ADED7ECCF17F0ECCF16F006
:10547000ECCF15F0ECCF14F0ECCF13F0ECCF12F032
:10548000ECCF11F0ECCF10F0120010C0EDFF11C006
:10549000EDFF12C0EDFF13C0EDFF14C0EDFF15C00E
:1054A000EDFF00C210F0116A1050126E1226113476
:1054B000136ED8901236133601C210F0116A1138EB
:1054C000F00B156E1038146E0F0B141A15261450AD
:1054D000121215501312F20E24EC16F07F0E121455
:1054E000106E116A105024EC16F012341334126E40
:1054F000136A1336129E125024EC16F0ECCF15F0FE
:10550000ECCF14F0ECCF13F0ECCF12F0ECCF11F0A5
:10551000ECCF10F012000001FCA508D0FC95FA0EAB
:1055200024EC16F00001FC810001F1810001FCA9CE
:1055300008D0FC99FB0E24EC16F00001FC9300014E
:10554000F1810001FCA70BD0FC97FC0E24EC16F0B7
:105550000001FC91FC930001FB6B0001F181000153
:10556000FB511CE0F80E24EC16F0F29E0001FB0744
:10557000F28E89EC1CF00001FE2BFE51180A0BE1A3
:105580000001FE6B0201002B0051040A04E102013C
:10559000006B0201012B0001F181E1D71200D9CF8C
:1055A000EDFFE9CFD9FF020EDBCFF7F0180E0001B7
:1055B000F86F2F0E0001F36FAF0E0001F46F080EAD
:1055C0000001F56F0001F66B010E0001F96F00019B
:1055D000F96BFA6B180EF86FF535F437F337FA37C5
:1055E000F937F537F751FA5FF651D8A0F63DF95F74
:1055F000D8B0F581F5B103D0F927F751FA27F82F84
:10560000EBD7F4C0F3FFF5511200F36AE86AECCF70
:10561000D9FF120010C0EDFF11C0EDFF12C0EDFF69
:1056200013C0EDFF14C0EDFF0001EF510001F003C6
:10563000F3CF10F0F4CF11F01050126E136A125025
:10564000D6240001EF6F1150126E146A690E1224F5
:105650000001F06F000EED6E3F0EED6EA40EB2EC89
:105660002CF0020EE926105092EC16F0ECCF14F05C
:10567000ECCF13F0ECCF12F0ECCF11F0ECCF10F038
:105680001200D9CFEDFFE9CFD9FF10C0EDFF11C057
:10569000EDFF020EDBCF10F08E0E88EC16F0000E40
:1056A000ED6E3F0EED6E9E0EB2EC2CF0020EE92672
:1056B000105092EC16F0B00E00018225116E1150C0
:1056C00024EC16F0000E24EC16F0105024EC16F02A
:1056D000ECCF11F0ECCF10F0ECCFD9FF1200000EA0
:1056E000ED6E3D0EED6E1E0E70EC2DF0020EE926F5
:1056F000100E78EC16F0010E80EC16F0000E7CEC2B
:1057000016F0080E36EC16F040EC16F0070E30ECF2
:1057100016F054EC25F00CEC2DF0780EED6EEAEC62
:105720002BF0E92AFFEC29F0240E00018A6F010E0C
:105730000001896F120082EC16F0000E88EC16F062
:10574000000EED6E3F0EED6E060EB2EC2CF0020E6A
:10575000E926400E88EC16F0000EED6E3F0EED6E61
:10576000140EB2EC2CF0020EE926800E88EC16F036
:10577000000EED6E3F0EED6E240EB2EC2CF0020E1C
:10578000E926B7EC29F0120010C0EDFF0001F1B1DD
:1057900001D01DD00001F191510E88EC16F04DECB6
:1057A0002EF0106E105092EC16F0100E88EC16F0E1
:1057B00000018529106E105090EC16F02F0E94EC1D
:1057C00016F002010029106E10508EEC16F0ECCF8E
:1057D00010F01200D9CFEDFFE9CFD9FF10C0EDFFD7
:1057E00011C0EDFF020EDBCF02F202010251ED6E9D
:1057F000CFEC2AF0106EF3CF11F0E92A1150ED6EC4
:105800001050ED6E030EBCEC2DF0020EE926ECCF2D
:1058100011F0ECCF10F0ECCFD9FF120010C0EDFF6B
:105820000001FCA107D0FCA302D0FC8914D0000128
:10583000FC8311D00001FCA302D0106A02D0010E3B
:10584000106E1050010BE844FE0BF46E0001FC5189
:10585000FD0BF410FC6F0001F181ECCF10F0120091
:10586000E9CFD9FF0A6EDCCFE1FFDCCFE2FFDC52EB
:10587000DCCF03F0DCCF04F0E6CF06F0E6CF07F094
:1058800010EE06F00A50DCEC16F0E9CFD9FFDCCFC1
:10589000E1FFDCCFE2FF06C0E6FF07C0E6FF120033
:1058A00010C0EDFF11C0EDFF106A0F0E105C0EE28C
:1058B000B00E1024116E115024EC16F07B0E24EC67
:1058C00016F0000E24EC16F0102AEFD7ECCF11F0F2
:1058D000ECCF10F01200D9CFEDFFE9CFD9FF020EC7
:1058E000DBCF8AF0510E88EC16F0000EED6E3F0E05
:1058F000ED6EA20EB2EC2CF0020EE92600018A51E8
:1059000090EC16F0ECCFD9FF12000001FDA112D0EF
:10591000FD9183888398838883988388839883887C
:1059200083988388839883888398838883988388DF
:10593000839801D083986CEC25F0120010C0EDFF25
:10594000E86A0001FCB1E82A106E105004E1E7ECAF
:105950002DF045EC2AF00001FC870001F181ECCF2D
:1059600010F01200F66EE9CFD9FFDCCFF7FFDCCFE5
:10597000F8FF0900F55003E094EC16F0FAD7120096
:1059800000000000000000000001240000000000F2
:105990000000000000000000000000018B6B9EEC86
:1059A0002CF00001876B0001866B0001856B50ECC9
:1059B0002CF012000201015101E001070001FE6B11
:1059C0000201006B45EC2AF00001F1811200F66E35
:1059D000E9CFD9FFDCCFF7FFDCCFF8FFDCCFE1FF69
:1059E000DCCFE2FFB4EF16F0F66EE9CFD9FFDCCFE3
:1059F000F7FFDCCFF8FFDCCFE1FFDCCFE2FFB6EF53
:105A000016F00201012B0001FE6B0201006B45EC58
:105A10002AF00001F1811200000E0001FC6F000E5F
:105A20000001FD6F0001FB6BE7EC2DF01200036E2F
:105A3000E9CFD9FFDCCF04F0DCCFE1FFDCCFE2FF20
:105A4000F2EF16F0036EE9CFD9FFDCCF04F0DCCF24
:105A5000E1FFDCCFE2FF18EF17F00001FCA106D058
:105A6000FCB304D00001FB2B0001FD811200E9CF43
:105A7000D9FFDCCFF8FFDCCFF7FFDCCFF6FF9CEFE0
:105A800016F0E9CFD9FF036EDCCF04F0DCCF05F0D0
:105A9000DC50A8EF16F0E9CFD9FFDCCFF6FFDCCF62
:105AA000F7FFDCCFF8FFE4EF16F0E7EC2DF045EC64
:105AB0002AF00001FC850001F1811200F66EE9CFA9
:105AC000D9FFDCCFF7FFDCCFF8FF9AEF16F0F66EC8
:105AD000E9CFD9FFDCCFF7FFDCCFF8FF9EEF16F060
:105AE000F66EE9CFD9FFDCCFF7FFDCCFF8FFE6EFAA
:105AF00016F0F66EE9CFD9FFDCCFF7FFDCCFF8FF69
:105B0000AAEF16F0A96EE9CFD9FFDCCFE1FFDCCF19
:105B1000E2FF1AEF17F0A96EE9CFD9FFDCCFE1FF62
:105B2000DCCFE2FF1CEF17F0E9CFD9FFDCCF03F0A9
:105B3000DCCF04F052EF16F0E9CFD9FFDCCF03F051
:105B4000DCCF04F074EF16F0E9CFD9FFDCCF03F01F
:105B5000DCCF04F0A4EF16F0036EE9CFD9FFDCCF61
:105B600004F0DC50BAEF16F0E9CFD9FFDCCF03F038
:105B7000DCCF04F0BCEF16F0E9CFD9FFDCCF03F0A7
:105B8000DCCF04F01EEF17F0D9CFEDFFE9CFD9FF3E
:105B9000ECCFD9FF1200D9CFEDFFE9CFD9FFECCF81
:105BA000D9FF1200D9CFEDFFE9CFD9FFECCFD9FF54
:105BB0001200D9CFEDFFE9CFD9FFECCFD9FF12000A
:105BC000D9CFEDFFE9CFD9FFECCFD9FF120000010B
:105BD000FE6B0201006B0201016B1200036EE9CF44
:105BE000D9FFDCCF04F0B8EF16F0010080590000B7
:105BF000800000001A000000E9CFD9FFDCCF03F0DD
:105C000060EF16F0E9CFD9FFDCCF03F068EF16F0B4
:105C1000E9CFD9FFDCCF03F06AEF16F0E9CFD9FF67
:105C2000DCCF03F06EEF16F0E9CFD9FFDCCF03F045
:105C300072EF16F0E9CFD9FFDCCF03F0F6EF16F0E4
:105C4000E9CFD9FFDCCF03F0F8EF16F0E9CFD9FFA9
:105C5000DCCF03F0AEEF16F0A96EE9CFD9FFDC5030
:105C6000B2EF16F0036EE9CFD9FFDC50F4EF16F077
:105C70009BEC2BF00001F18112008CEC25F08BECF9
:105C80002AF012003AEC16F004C0F3FF120076EC92
:105C900025F012002DEC2DF012000201025112002D
:0C5CA000A96EB0EF16F0A6EF16F012008F
:00000001FF
